:020000040000FA
:020000001728BF
:08000800A3000230A20A22024B
:10001000031D1528122823080030A2032207031D00
:1000200015281228A201230826282308262883162B
:100030000030870000308600033085008312A20163
:100040002628A00B21286430A000080005180428E9
:1000500085180B282F2022084920870026280030E9
:100060002202031941200130220203193B203920CA
:100070000800061608000612212006162120061286
:100080000800061221202120212006162120061218
:0C0090000800820706345B344F3408007F
:02400E00D430AC
:00000001FF
